:1000000012C018951895189518951895D1C6189579
:100010001895189518951895189518951895189578
:100020001895189518958FE58DBFC0EEE8EF4E2E08
:1000300084E08EBFD3E0F2E05F2EEEEFF3E0A0E6C7
:10004000B0E0A89584B7082E877F84BF88E1992700
:1000500081BD91BD88278D933197E9F76624EED74E
:100060008AD423D000917300013009F01DC080E0D4
:100070008093730000917900013B09F002C0BAD46B
:1000800013C0023B09F002C0FAD20EC0043B09F0D3
:1000900002C06FD109C0063B09F002C058D004C0AD
:1000A000073B09F001C001D1DDCFEBD7F8D687E0DF
:1000B00080937A0080E080937B00ACE7B0E0EEE5CF
:1000C000F9E18CDBEED78AE180937A0080E08093BF
:1000D0007B00ACE7B0E0E0E7F9E180DBADEDB0E05C
:1000E000E8E8F9E17BDBA5EFB0E0E8E8F9E176DBF1
:1000F0007FD88EE280937A0080E080937B00ACE72B
:10010000B0E0E0EAF9E16ADBADE0B1E0E6EBF9E1AD
:1001100065DBA5E2B1E0E6EBF9E160DB69D882E4FA
:1001200080937A0080E080937B00ACE7B0E0ECEC59
:10013000F9E154DBADE3B1E0E4EEF9E14FDBA5E535
:10014000B1E0E4EEF9E14ADB53D895D6089599D7AA
:10015000A6D682E480937A0080E080937B00ACE7AF
:10016000B0E0ECEFF9E13ADBADE3B1E0E4E1FAE174
:1001700035DBA5E5B1E0E4E1FAE130DB39D884E232
:1001800080937A0080E080937B00ACE7B0E0ECE203
:10019000FAE124DBA5EFB0E0E6E3FAE11FDBADE036
:1001A000B1E0E6E3FAE11ADB23D880E180937A003C
:1001B00080E080937B00ACE7B0E0E0E4FAE10EDBA6
:1001C000A5ECB0E0E8E4FAE109DBADEDB0E0E8E48D
:1001D000FAE104DB0DD888E380937A0080E0809315
:1001E0007B00ACE7B0E0E0E5FAE1F8DAA5E2B1E0E7
:1001F000E8E5FAE1F3DAADE3B1E0E8E5FAE1EEDAF9
:10020000F7D739D600917300013009F047C08AE171
:1002100080937A008AE080937B00ACE7B0E0E0E670
:10022000FAE1DCDA8CE6482F00917900041709F036
:1002300006C0ACE7B0E0EEE6FAE1D0DA2BC082E728
:10024000482F041709F006C0ACE7B0E0ECE7FAE18C
:10025000C5DA20C08FE6482F041709F006C0ACE7C6
:10026000B0E0EAE8FAE1BADA15C085E7482F0417EA
:1002700009F006C0ACE7B0E0E8E9FAE1AFDA0AC09D
:1002800082E5482F041709F005C0ACE7B0E0E6EAC4
:10029000FAE1A4DA06D780E0809373000091790038
:1002A000053B09F0AFCF01DF0895EBD6F8D584E226
:1002B00080937A0080E080937B00ACE7B0E0E4EBD1
:1002C000FAE18CDAA5EFB0E0ECECFAE187DAADE028
:1002D000B1E0ECECFAE182DA8BD7CDD580E0809307
:1002E0007101AFE6B1E083DAAFE6B1E00D911C91A8
:1002F000063450E0150714F009F034C080916F0106
:1003000080937A0081E080937B00ADE6B1E06FDA04
:10031000ADE6B1E00D911C910F3050E0150710F0E3
:1003200009F013C0A1E7B1E08C91ACE7B0E08D9388
:1003300088278C93A1E7B1E08C918F5F8C93B1D625
:10034000ADE6B1E0E2D908F4E3CFAFE6B1E00D915C
:100350001C914AE050E0040F151FAFE6B1E00D9389
:100360001C93C2CF00917900053B09F0FBCF9DDEC5
:10037000089587D694D581E080937A0080E08093B9
:100380007B00ACE7B0E0E4EEFAE128DAECE7F0E07D
:10039000ADEAB0E0B6DA85D68BE080937A0080E0F3
:1003A00080937B00ACE7B0E0ECEFFAE117DAECE722
:1003B000F0E0A5ECB0E0A5DA74D685E180937A0090
:1003C00080E080937B00ACE7B0E0E4E1FBE106DA9B
:1003D000ECE7F0E0ADEDB0E094DA63D68FE1809326
:1003E0007A0080E080937B00ACE7B0E0ECE2FBE1D8
:1003F000F5D9ECE7F0E0A5EFB0E083DA52D689E278
:1004000080937A0080E080937B00ACE7B0E0E4E486
:10041000FBE1E4D9ADE0B1E0E4E4FBE1DFD941D6B2
:1004200083E380937A0080E080937B00ACE7B0E0C8
:10043000ECE5FBE1D3D9ECE7F0E0A5E2B1E061DA6D
:1004400030D68DE380937A0080E080937B00ACE728
:10045000B0E0E4E7FBE1C2D9ECE7F0E0ADE3B1E006
:1004600050DA1FD688E380937A0082E180937B0084
:10047000ACE7B0E0ECE8FBE1B1D9BAD687E4809311
:100480007A0080E080937B00ACE7B0E0E0E9FBE13C
:10049000A5D9ECE7F0E0A5E5B1E033DA02D6EBD47C
:1004A00083E380937A0082E080937B00ACE7B0E046
:1004B000E8EAFBE193D9ACE7B0E06BD9EBE6F0E01A
:1004C000BBD9ACE7B0E065D9EEEAFBE187D9ACE790
:1004D000B0E05FD9ECE6F0E0AFD9E3D58DE38093EF
:1004E0007A0082E080937B00ACE7B0E0E6EBFBE1D2
:1004F00075D9ACE7B0E04DD9EDE6F0E09DD9ACE7B9
:10050000B0E047D9ECEBFBE169D9ACE7B0E041D909
:10051000EEE6F0E091D9C5D589E180937A0083E1D8
:1005200080937B0000917400013010F009F001C04D
:1005300007C087E0ACE7B0E08D9388278C9306C0B6
:1005400086E0ACE7B0E08D9388278C93AAD5009124
:100550007300013009F08CC085E180937A0082E05D
:1005600080937B00ACE7B0E0E2ECFBE137D9ACE78D
:10057000B0E00FD9E8E7F0E05FD9ACE7B0E009D927
:10058000ECECFBE12BD9ACE7B0E003D9E7E7F0E016
:1005900053D9ACE7B0E0FDD8E0EDFBE11FD981D540
:1005A0008FE180937A0082E080937B00ACE7B0E03B
:1005B000E6EDFBE113D9ACE7B0E0EBD8E6E7F0E01D
:1005C0003BD9ACE7B0E0E5D8ECECFBE107D9ACE710
:1005D000B0E0DFD8E5E7F0E02FD9ACE7B0E0D9D85C
:1005E000E0EDFBE1FBD85DD5ACE7B0E0EEEDFBE183
:1005F000F5D8A9E7B0E08C91ACE7B0E08F93C9D80B
:100600008F918D9388278C93ACE7B0E0C2D8E4EE4D
:10061000FBE1E4D8ACE7B0E0BCD8E9E7F0E00CD906
:10062000ACE7B0E0B6D8E0EDFBE1D8D88BE0809342
:100630007A0082E080937B0034D5ACE7B0E0ECEE4A
:10064000FBE1CCD8ACE7B0E0A4D8E9E7F0E03ED9D4
:10065000ACE7B0E09ED8EAEFFBE1C0D889E2809336
:100660007A0082E080937B001CD580E08093730049
:1006700000917900053B09F04FCF17DD089501D5B2
:100680000ED485E180937A0080E080937B00ACE714
:10069000B0E0ECEFFBE1A2D8ECE7F0E0ADEDB0E0CC
:1006A00030D9FFD48FE180937A0080E080937B0083
:1006B000ACE7B0E0E4E1FCE191D8ECE7F0E0A5EFD5
:1006C000B0E01FD9EED489E280937A0080E0809375
:1006D0007B00ACE7B0E0ECE2FCE180D8ECE7F0E0D6
:1006E000ADE0B1E00ED9DDD483E380937A0080E001
:1006F00080937B00ACE7B0E0E4E4FCE16FD8ECE78A
:10070000F0E0A5E2B1E0FDD8CCD482E480937A0099
:1007100080E080937B00ACE7B0E0ECE5FCE15ED8E4
:10072000ADE3B1E0E4E7FCE159D8A5E5B1E0E4E7E9
:10073000FCE154D85DD58DE380937A0080E080930E
:100740007B00ACE7B0E0ECE8FCE148D8AAD493D356
:10075000A4E9B0E0E4E9FCE141D881E08093AC0099
:1007600087E480937A0080E080937B00E4E9F0E006
:10077000ACE7B0E0C6D8ACE7B0E00BD8E6E9FCE106
:100780002DD88FD400917300013009F0EDC0009195
:100790007900003808F023C0ACE7B0E0E8E9FCE1FC
:1007A0001DD8A9E7B0E08C91ACE7B0E08F93F1D70A
:1007B0008F918D9388278C93ACE7B0E0EAD7E4EE75
:1007C000FBE10CD8ACE7B0E0E4D7E9E7F0E07ED895
:1007D000ACE7B0E0DED7EAEFFBE100D822C0ACE73F
:1007E000B0E0E2EAFCE1FAD7A9E7B0E08C91ACE72F
:1007F000B0E08F93CED78F918D9388278C93ACE701
:10080000B0E0C7D7E4EEFBE1E9D7ACE7B0E0C1D791
:10081000E9E7F0E05BD8ACE7B0E0BBD7EAEFFBE19B
:10082000DDD78BE080937A0080E080937B0039D421
:1008300081E080937A0080E080937B00ACE7B0E0B9
:10084000ECEAFCE1CBD7ACE7B0E0A3D7E8E7F0E017
:10085000F3D7ACE7B0E09DD7EAEBFCE1BFD7ACE75C
:10086000B0E097D7E7E7F0E0E7D7ACE7B0E091D7A3
:10087000E0ECFCE1B3D715D400917900013080E0C1
:1008800010F009F081E08F9300917900003881E049
:1008900008F080E09F9189238F930091AC000C3089
:1008A00081E008F080E09F918923882309F42FC01C
:1008B000A9E7B0E08C91A4E9B0E08F936AD78F915B
:1008C0008D9388278C93ACEAB0E08C918F5F8C93EA
:1008D00087E480937A0080E080937B000091AC00F5
:1008E0000C3010F009F001C006C0E4E9F0E0ACE71C
:1008F000B0E007D80BC0E4E9F0E0ACE7B0E001D825
:10090000ACE7B0E046D7E6E9FCE168D7CAD300918E
:100910007900033B09F025C00091AC00013010F0D4
:1009200009F001C01EC08091AC0081508093AC00E2
:10093000E4E9F0E00091AC00A4E9B0E0E7D787E497
:1009400080937A0080E080937B00E4E9F0E0ACE7FC
:10095000B0E0D7D7ACE7B0E01CD7E4ECFCE13ED781
:10096000A0D380E08093730000917900053B09F0EB
:1009700009CF9BDB089582E390E021D772D38AE010
:1009800090E01DD774D37DD3E3D22EE42BBD2FE1AD
:100990002ABD2AE02EBD20E129BF789401D0089518
:1009A000E0E0F0E0ADE6B1E092E0D2D7ADE6B1E054
:1009B0000D911C910D3A50E0150709F019C0E2E0C5
:1009C000F0E0ABE6B0E091E0C3D7E3E0F0E0ACE606
:1009D000B0E091E0BDD7E4E0F0E0ADE6B0E091E05A
:1009E000B7D7E5E0F0E0AEE6B0E091E0B1D701C006
:1009F00001D0089546D353D2A5D000916D0002379F
:100A000081E008F080E08F9300916D00023880E073
:100A100010F009F081E09F91892B882309F402C02E
:100A200057D054C000916E00023581E008F080E09C
:100A30008F9300916E00023680E010F009F081E0A3
:100A40009F91892B882309F402C042D03FC00091B6
:100A50006B00063480E010F009F081E08F93009184
:100A60006C00053580E010F009F081E09F91892B42
:100A7000882309F402C02CD029C08DEA90E0ADE6AD
:100A8000B1E08D939C93E0E0F0E0ADE6B1E092E060
:100A90007BE74DD7E2E0F0E0ABE6B0E091E07BE74A
:100AA00046D7E3E0F0E0ACE6B0E091E07BE73FD78B
:100AB000E4E0F0E0ADE6B0E091E07BE738D7E5E0D8
:100AC000F0E0AEE6B0E091E07BE731D7EEDA0895F2
:100AD00083E380937A0081E080937B00ACE7B0E011
:100AE000E8ECFCE17BD6ACE7B0E053D6EDE6F0E015
:100AF000A3D6ACE7B0E04DD6E4E9FCE16FD6D1D2A5
:100B0000ACE7B0E0ECECFCE169D6ACE7B0E041D694
:100B1000EEE6F0E091D6C5D2ACE7B0E0E0EDFCE166
:100B20005DD6BFD28AE780936D008AE580936E0020
:100B300081E380936B0081E480936C00E5E0F0E05A
:100B40002FD60895ACE7B0E0E8EDFCE147D68FE1A1
:100B500080937A0085E080937B00A3D2ACE7B0E07D
:100B6000E8EEFCE13BD68DE280937A0085E080934D
:100B70007B0097D2E1E0F0E013D681E0ACE7B0E093
:100B80008D9388278C9382E0ACE7B0E08F9301D6F9
:100B90008F918D9388278C9386E080937A0080E0F4
:100BA00080937B00FAD080917500809363008091E0
:100BB00076008093670086E080937A0085E18093D9
:100BC0007B00EBD08091750080936400809176006B
:100BD0008093680082E480937A0080E080937B00B9
:100BE000DCD08091750080936500809176008093C1
:100BF000690082E480937A0085E180937B00CDD008
:100C000080917500809366008091760080936A00E1
:100C1000A3E6B0E00D911127A5E6B0E04D91552770
:100C2000040F151FADE6B1E00D931C93ADE6B1E0E6
:100C30000D911C9141E050E0040F151FADE6B1E0AD
:100C40000D931C93ADE6B1E00D911C9142E050E094
:100C500086D5ADE6B1E04D935C9380916D018093B4
:100C60006B00A8E6B0E00D911127A7E6B0E04D912A
:100C70005527040F151FADE6B1E00D931C93ADE6AB
:100C8000B1E00D911C9141E050E0040F151FADE65D
:100C9000B1E00D931C93ADE6B1E00D911C9142E0E3
:100CA00050E05DD5ADE6B1E04D935C9380916D0170
:100CB00080936C00A4E6B0E00D911127A3E6B0E0AC
:100CC0004D915527041B150BADE6B1E00D931C9318
:100CD000A6E6B0E00D911127A5E6B0E04D915527AD
:100CE000041B150BAFE6B1E00D931C93ADE6B1E02C
:100CF0000D911C91AFE6B1E04D915C91040F151F71
:100D0000ADE6B1E00D931C930AE718EAADE6B1E059
:100D10004D915C9124D5ADE6B1E04D935C9380910B
:100D20006D0180936D00AAE6B0E00D911127A8E651
:100D3000B0E04D915527041B150BADE6B1E00D93C6
:100D40001C93A9E6B0E00D911127A3E6B0E04D9108
:100D50005527041B150BAFE6B1E00D931C93ADE6D0
:100D6000B1E00D911C91AFE6B1E04D915C91040FA3
:100D7000151FADE6B1E00D931C9300E915E6ADE655
:100D8000B1E04D915C91EBD4ADE6B1E04D935C9355
:100D900080916D0180936E00089583D1009173005E
:100DA000013009F0FBCF80E0809373006AD1089591
:100DB0000F921F922F923F924F925F927F92AF922B
:100DC000BF920F931F932F933F934F935F936F9314
:100DD0007F938F939F93AF93BF93CF93DF93EF93C3
:100DE000FF938FB78F93AFE6B0E08C918F5F8C93BA
:100DF00000916F00023309F003C080E080936F0020
:100E0000A0E7B0E08C918F5F8C930091710000306F
:100E100010F009F001C005C08091710081508093ED
:100E2000710000917200003010F009F001C005C09F
:100E300080917200815080937200A8D08F918FBFF3
:100E4000FF91EF91DF91CF91BF91AF919F918F91E2
:100E50007F916F915F914F913F912F911F910F91D2
:100E6000BF90AF907F905F904F903F902F901F90DA
:100E70000F901895E2C020ECADEAB0E03D91383219
:100E800059F43C9130683E933D933D932A9531F05F
:100E90004C913D934932D1F72A9581F7089520EC82
:100EA0003327ADEAB0E03D932A95E9F7089533275B
:100EB0001124A6E7B0E00C903324ACE6B0E02C900F
:100EC000021813086AF0202CAEE6B0E03C90239C98
:100ED0001694169416941394312D383008F037E098
:100EE000A8E7B0E03C9333271124A5E7B0E00C90CD
:100EF0003324ABE6B0E02C900218130862F0202CEB
:100F0000ADE6B0E03C90239C169416941394312DDA
:100F1000373108F036E1A7E7B0E03C93A8E7B0E04E
:100F20002C912395ADEAB0E02A9511F05896FCCFAC
:100F30001124A30FB11D2C91203209F422272F3543
:100F400011F420E201C0D2D0A9E7B0E02C930895BB
:100F500014D00ED020E0A0E6B0E02C93A1E6B0E0E3
:100F60002C93A4E7B0E02C93A3E7B0E02C93089572
:100F700020E627B927E826B90895A09AA19AA29A4F
:100F8000A39AA89AA99AAB9AAA9A0895A4E7B0E05E
:100F90000C91A3E7B0E01C91A298A398A89823E62F
:100FA00027B941D0A6E7B0E01C92A198A098AB98D1
:100FB00020E627B938D0A5E7B0E01C92A5E7B0E05D
:100FC0002C91203F40F5A6E7B0E02C91203F18F58A
:100FD00001FD22C0A5E7B0E02C91A0E6B0E03C9175
:100FE000231761F4A6E7B0E02C91A1E6B0E03C91B4
:100FF000231721F4026011605ADF0EC0A5E7B0E0AC
:101000002C91A0E6B0E02C93A6E7B0E02C91A1E6ED
:10101000B0E02C9301C00D7FA3E7B0E01C93A4E7E0
:10102000B0E00C930895369A3699FECF369A3699E9
:10103000FECF002415B0A1DF0895D9C08A988B98FF
:101040008C988E988F98929A939A949A969A979A47
:101050008A9A8B9A8C9A8E9A8F9A9498969A979A43
:10106000089597982FEF2A95F1F7979A0895EAEF48
:10107000F2E1259125916591559172D02A95D9F784
:1010800008956AE050E06CD06BE050E069D06CE00D
:1010900050E03AE028EC64D02A95E9F73A95D1F788
:1010A0000895ACE7B0E0EAE7F0E0008038E1A32E75
:1010B000132E019CEBE7F0E080819927800D911DB4
:1010C0002D9114D0B22E4FE7B42279F048E0042ECF
:1010D00011240B9CEAE0F3E1E00DF11D25D0EBE7D4
:1010E000F0E0308133953083EBCF089527FF1BC0AC
:1010F000243C11F42BE517C0263D11F42CE513C058
:101100002C3D11F42DE50FC0243E11F42BE70BC04C
:10111000263F11F42CE707C02C3F11F42DE703C044
:101120002F3D09F42EE70895082E192E01969924D3
:1011300028E1A22E28E06AE0502D12D06BE0512D5C
:101140000FD045913AE0441F57953A95E1F708F4DE
:1011500050646CE005D00A0C191C2A9561F70895BB
:101160002F9396980AC09498000000000000000099
:1011700000000000000000000000949A0000000041
:101180000000000000000000B799EDCF0000949827
:1011900093980000000000002FEF27BB000068BB01
:1011A0000000949A00000000000000000000000011
:1011B0000000000000009498000000000000000003
:1011C0000000929858BB0000949A000000000000B4
:1011D00000000000000000000000000094980000E3
:1011E000969A20E027BB939A929A2F91089583C0F4
:1011F000ACE7B0E0E2E7F1E044272D91233209F4B7
:101200002DE02F3509F42CE02C3309F428E02E339F
:1012100009F429E0243209F42AE0263209F42BE00B
:10122000208F203071F1283211F4332703C02B3581
:1012300061F438E041E024E1230F20AB23E1230FE8
:10124000208F20E1230F2193D8CF293211F02D35A3
:1012500059F4442726E1230F20AB27E1230F208FE9
:1012600022E1230F2193C9CF413039F425E1230F27
:1012700020AB21E1230F2193C0CF20E220AB2193AB
:10128000BCCF22272083208F20ABEBE7F0E020812A
:10129000EBEBF1E02083EAE7F0E02081EAEBF1E01C
:1012A0002083265027FD2227EAE7F0E02083A2E7EB
:1012B000B1E0F9DEEBEBF1E02081EBE7F0E0208339
:1012C000EAEBF1E0208136E0230FEAE7F0E020834B
:1012D000A2EAB1E0E8DEEBEBF1E02081EBE7F0E041
:1012E0002083EAEBF1E02081EAE7F0E02083AAE83E
:1012F000B1E0D9DE0895F894FFCF0007001201761F
:101300000217034F0800090000320000000000002F
:10131000000000000047000000002020201E2020C8
:101320002000000F11110A0A1B00303007080808BE
:1013300007000001010202140800000F5050500F76
:101340000000000F5F5F5F0F000003070F1F0F0714
:101350000300181C1E1F1E1C1800007F7F1F0E0498
:10136000000000040E1F3F7F0000003F4044481F64
:101370000804404448507F100804030D0B0D0B1B5C
:10138000180000150E1B0E150000004F1010101055
:101390001010007F000000000000003E010101016C
:1013A000010110101010101010101010101010105B
:1013B0004F000000000000007F000001010101015A
:1013C0003E000101010101010101004F5F1C1C1CD5
:1013D0001C1C007F7F0000000000003E3F07070745
:1013E00007071C1C1C1C1C1C1C1C1C1C1C1C1C5F24
:1013F0004F0000000000007F7F0000070707073F45
:101400003E00070707070707070700000000000066
:101410000000040E0E04040004001B1B1200000058
:101420000000000A1F0A0A1F0A00080E100C021C06
:1014300004001919020408131300081414081512E3
:101440000D000C0C08000000000004080808080843
:1014500004000804040404040800000A0E1F0E0A15
:1014600000000004041F0404000000000000000C41
:101470000C080000001F0000000000000000000C2D
:101480000C0000010204081000000E1113151911C0
:101490000E00040C040404040E000E1101060810D2
:1014A0001F000E11010E01110E0002060A121F028A
:1014B00002001F10101E01110E000608101E11114F
:1014C0000E001F010204080808000E11110E111170
:1014D0000E000E11110F01020C0000000C0C000C8C
:1014E0000C0000000C0C000C0C080204081008048E
:1014F000020000001F00001F000008040201020497
:1015000008000E110106040004000E111715171033
:101510000E000E1111111F1111001E11111E1111BB
:101520001E000E11101010110E001E1111111111BC
:101530001E001F10101E10101F001F10101E101074
:1015400010000E11101711110F001111111F1111A0
:1015500011000E04040404040E0001010101111124
:101560000E00111214181412110010101010101087
:101570001F00111B15111111110011191513111153
:1015800011000E11111111110E001E11111E10105B
:1015900010000E11111115120D001E11111E121145
:1015A00011000E11100E01110E001F04040404049A
:1015B00004001111111111110E0011111111110A54
:1015C00004001111151515150A0011110A040A114C
:1015D00011001111110A040404001E020408101065
:1015E0001E0011040A111F11110011000E1111111A
:1015F0000E001100111111110F00040A110000005A
:1016000000000000000060607F000C0C040000007F
:10161000000000000E010F110F0010101E1111111B
:101620001E0000000E1110110E0001010F1111110A
:101630000F0000000E111E100E000608081E0808FC
:10164000080000000F11110F010E10101C121212D1
:101650001200040004040404060002000602020250
:10166000120C1010121418141200040404040404C0
:10167000060000001A151511110000001C121212AC
:10168000120000000E1111110E0000001E111111A8
:101690001E1000000F1111110F010000160908089B
:1016A0001C0000000E100E010E0000081E08080AA3
:1016B00004000000121212160A0000001111110A93
:1016C000040000001111151F0A00000012120C1274
:1016D000120000001212120E041800001E020C105C
:1016E0001E000A000E010F110F000A00000E11115A
:1016F0000E000A00001111110E000C121412111E1E
:101700001000040E1B11111F0000ED91FC91EF5F02
:10171000FF4FFC93EE93089500FC10D0089503D082
:101720001ED001F8F9CF0024E89457FF02C009D079
:10173000689400F80BD010F80124089502D009D065
:101740000895509540954F5F5F4F0895E89417FFB7
:101750000895009510950F5F1F4F68940895352FD9
:10176000242FE894452B11F468940895512F402FAD
:101770000027112780E1440F551F001F111F021B76
:10178000130B416018F4020F131F4E7F8A9599F7CF
:1017900008958F938D918823E9F711978F9108957C
:1017A00088EE93E00CD03197D9F708953197F1F78F
:1017B0000895689462F80895E89462F80895EF93A4
:1017C000FF93EE27E82BE92B31F0E0EDF7E03197BE
:1017D000F1F70197D1F7FF91EF91089504D00D92A1
:1017E0000020E1F70895C89531960020089582E021
:1017F00001C084E099279D938A95E9F70895000F29
:10180000111F221F331F08950095109520953095C4
:101810000F5F1F4F2F4F3F4F0895019110810EC052
:1018200001911191219130810BC00191108117FF1D
:1018300005C03FEF2FEF04C0008111272227332777
:1018400037FF03C0E1DF8DE28D93CF93DF93CF921B
:10185000DF92EF92AA24BB24CC24DD24EE2440E2C4
:10186000CAE0DD2755E093E38881890F87FD9F70EB
:1018700083FD907F891B89935A95A9F7C0DFAA1C25
:10188000BB1CCC1CDD1CEE1C4A9551F7E894EFE024
:10189000FF2782910ED0EB30E0F71EF068948A2D7E
:1018A0000CD088278D93EF90DF90CF90DF91CF9170
:1018B0000895982F829501D0892F8F70805D26F032
:1018C000803309F4089568948D93089541E003C02E
:1018D00042E001C044E0E40F8827F81F8291982F6E
:1018E000829505D0892F03D04A95C1F707C08F7024
:1018F0008A3008F0895F805D8D93089588278D93E5
:10190000089581918D938823E1F7089581918D93B6
:101910000A9519F08823D1F70895F0CFE199FECF09
:10192000EEBBFFBB3196089591E001C092E07B379A
:1019300051F47FB7F894F2DF8D918DBBE29AE19A72
:101940009A95C9F77FBF7727089591E001C092E08B
:10195000E5DFE09A8DB38D939A95D1F70895202015
:1019600020204120552053205720412048204C0062
:10197000284368722D4C69737465202928546F754B
:101980006368746573742900283720202020202084
:101990002020202928342020202020202020290039
:1019A00020202853796D626F6C6520616E7A6569BD
:1019B00067656E2900002020283620202020202066
:1019C0002020202020202020202900002028204B1B
:1019D000616C2E2920202020202028205465787436
:1019E000202900002028312020202029202020200C
:1019F0002020283220202020202900002020202004
:101A00002020202020202020202028232920205B87
:101A10005F5D00002020202020202020202020208A
:101A200020205252522020283529000020283C290D
:101A300020283E290000206C6C6C2072727200001D
:101A400020202028262900002020206F6F6F000012
:101A500020202028242900002020207575750000F2
:101A600020202020202020202020202000006E6127
:101A70006368206C696E6B73202000006E61636880
:101A8000207265636874732000006E616368206F64
:101A900062656E20202000006E61636820756E74A0
:101AA000656E2020000052657475726E73796D62E8
:101AB0006F6C0000202020202020202020202020CB
:101AC000202020202020205B5F5D0000202020209F
:101AD00020202020202020202020202020202028FE
:101AE000352900003031323334353637383930312A
:101AF0003233343536373839303132003120202016
:101B000020202020202020202020202020202020D5
:101B10002020C4003220202020202020202020202F
:101B200020202020202020202020D600332020200C
:101B300020202020202020202020202020202020A5
:101B40002020DC00342020202020202020202020E5
:101B500020202020202020202020E40035202020CC
:101B60002020202020202020202020202020283558
:101B70002920F60036202020202020202020202090
:101B800020202020202028352920FC005B5F5D00DC
:101B9000376162636465666768696A6B6C6D6E6FF6
:101BA000707172737475DF005831503D0000202051
:101BB0005931503D00005870533D00002059705A73
:101BC0003D005261737465723A593D0020583D00E2
:101BD0002020202000004665696E3A593D00436888
:101BE000723A000020576572743D000052FC636B2E
:101BF00067616265776572743A006800204142430C
:101C00004445464748494A4B4C4D4E4D4F50203174
:101C100032332000205152535455565758595AC404
:101C2000D6DC20202020203435360000206162637D
:101C30006465666768696A6B6C6D6E6F70202037CB
:101C400038390000207172737475767778797AE488
:101C5000F6FCDF2020202030205F00002020202004
:101C6000202020202020202020202844454C2920EE
:101C70005B5F5D00202020202020202020202020CD
:101C800020202833202029202835290020496E7063
:101C900075743A0020002D005A65696368656E20EE
:101CA0003A0046756E6B74696F6E3A00506F7369D7
:101CB00074696F6E3A2020593D002020583D000085
:101CC000202020002D2000004B583D004B593D00A6
:101CD000204665686C6572005A756D204B616C69B1
:101CE0006272696572656E004B7265757A65206116
:081CF0006E74697070656E00EE
:00000001FF
